:020000040000FA
:04000000B2EF01F06A
:0400080038EF12F0CB
:0800180091EF12F00F0BAB6F2A
:10002000000EF76E360EF66EAB51F626D8B0F72AF4
:100030000800F55012003031323334353637383954
:10004000414243444546000EF86E2A0EF76E7C0E80
:10005000F66EE3EC11F0000EF86E2A0EF76E8E0EBF
:10006000F66EE3EC11F073EC10F012D0000EF86EA7
:100070002A0EF76E580EF66EE3EC11F0000EF86ED5
:100080002A0EF76E6A0EF66EE3EC11F06FEC10F0CC
:10009000476A486A0882120002D87BEC10F0D58EBD
:1000A0007BEC10F0D59E8A961200FF0EBB6E0C0EF4
:1000B000BD6E496A4A6A10D80C0E666E4B6A4C6A6D
:1000C00028D8000EBA6E030EBC6EBA841200496ABC
:1000D0004A6A05D88C94120043A0F9D78C84040096
:1000E00049C0A6F04AC0A7F0D890A733A633D8904D
:1000F000A733A633A6C0BEFFBD98BD9A49B0BD8840
:1001000049B2BD8A1200E3DF4B6A4C6A05D88B986E
:10011000120043A2F9D78B8804004BC0A6F04CC054
:10012000A7F0D890A733A633D890A733A633A6C09C
:1001300067FF6698669A4BB066884BB2668A120073
:10014000430E3B6EE10E3A6E376A386A396AABECA1
:1001500015F0450E3B6EC80E3A6EE00E396E376AEA
:10016000386A04EC1AF032C058F033C059F034C089
:100170005AF035C05BF036C05CF01200240E056EFC
:1001800020EE9CF0050EA66F27EC12F079EF10F030
:10019000240E056E20EE9CF0050EA66F30EF12F0D7
:1001A000220E056E20EE9AF0020EA66F27EC12F0DA
:1001B00079EF10F0220E056E20EE9AF0020EA66F77
:1001C00030EF12F0210E056E20EE46F0010EA66F04
:1001D00027EC12F079EF10F0210E056E20EE46F0BC
:1001E000010EA66F30EF12F0200E056E20EE45F0E6
:1001F000010EA66F27EC12F079EF10F0200E056EBD
:1002000020EE45F0010EA66F30EF12F0290E056EBC
:1002100020EE43F0010EA66F27EC12F079EF10F0FC
:10022000290E056E20EE43F0010EA66F30EF12F09E
:100230001F0E056E20EE07F0010EA66F27EC12F0E0
:1002400079EF10F01F0E056E20EE07F0010EA66F7D
:1002500030EF12F01C0E056E20EEB4F0020EA66F09
:1002600027EC12F079EF10F01C0E056E20EEB4F0C2
:10027000020EA66F30EF12F01A0E056E20EEB0F0EF
:10028000020EA66F27EC12F079EF10F01A0E056E31
:1002900020EEB0F0020EA66F30EF12F0140E056ED5
:1002A00020EE94F0050EA66F27EC12F079EF10F017
:1002B000140E056E20EE94F0050EA66F30EF12F0CE
:1002C000190E056E20EE99F0010EA66F27EC12F0C4
:1002D00079EF10F0190E056E20EE99F0010EA66F61
:1002E00030EF12F0000E056E20EE80F0140EA66FB7
:1002F00027EC12F079EF10F0000E056E20EE80F082
:10030000140EA66F30EF12F0C7EC11F0000EF86E6D
:100310002A0EF76E340EF66EE3EC11F0000EF86E56
:100320002A0EF76E460EF66EE3EC11F0FFD7C7EC1F
:1003300011F0000EF86E290EF76EF20EF66EE3EC79
:1003400011F0000EF86E2A0EF76E040EF66EE3EC56
:1003500011F082EC15F0BFC01DF0D6EC1FF0B5EC2B
:100360001EF0120094EC10F0D0B60FD083EC00F029
:100370000886BF2BDCDF0A0EA66F4CEC00F0A62F20
:10038000FCD7C7EC11F0088204D0D3EC10F0DAEC03
:1003900010F055EC00F07CEC01F022EC01F06AEC7E
:1003A00001F058EC01F046EC01F034EC01F0FEEC09
:1003B00000F0ECEC00F0DAEC00F0C8EC00F010EC2F
:1003C00001F079EC10F0A0EC00F04F8A508A5768E9
:1003D000B0C0AEF0B1C0AFF0B4C0B2F0B5C0B3F0D1
:1003E000C80EB76FC80EB86F83EC00F008A6DFEC3C
:1003F00004F0C80EB96FC80EBA6F4FEC00F00400DD
:10040000F7EC0FF0D8A08EEF02F083EC00F011ECC7
:1004100010F0425206E0426AC7EC11F06FEC10F0A7
:1004200075D0010E476203D0010E996F0BD0020EFA
:10043000476203D0020E996F05D0030E476211D0B8
:10044000030E996F60EC01F007B40BD0D00EBB6FB8
:10045000070EBC6FD00EBD6F070EBE6F449244985E
:1004600055D0040E47621AD008A416D0089450C183
:1004700099F04BC143F0A1C01DF0D2EC17F02DC094
:1004800094F02EC095F02FC096F030C097F031C098
:1004900098F04EEC01F03AD05BEC05F0050E4762A7
:1004A00003D09FEC04F0996B0B0E476206D04370AB
:1004B0008DEC05F006EC01F029D00C0E476206D059
:1004C00043728DEC05F006EC01F020D00D0E476272
:1004D0000BD0000EF86E250EF76EFE0EF66EE3ECF6
:1004E00011F06FEC10F012D00E0E476202D04AEC01
:1004F00006F00F0E47620AD0000EF86E260EF76E59
:10050000220EF66EE3EC11F06FEC10F0C80EB96F2E
:10051000C80EBA6FC7EC11F00882476A4852D8B4C7
:1005200040D008A414D048AEA12B48BEA107A1C05A
:100530001DF0D2EC17F02DC094F02EC095F02FC016
:1005400096F030C097F031C098F0486A2AD099539D
:1005500003E09FEC04F0996B7BC032F07CC033F079
:100560007DC034F07EC035F07FC036F0400E3B6E6B
:10057000A00E3A6E376A386A396A48AE47EC1AF00C
:1005800048BE41EC1AF005EC17F032C07BF033C0E6
:100590007CF034C07DF035C07EF036C07FF0576807
:1005A000486A4F4E4F8A010E4F6200D0020E4F62D2
:1005B0002CD0504E508A010E506205D008A203D0B4
:1005C00063EC0EF00892020E506203D043B242EC8C
:1005D0000DF0030E506203D043B22FEC0DF0040E69
:1005E000506203D043B010EC0DF0050E506202D003
:1005F000FDEC0CF0060E506202D061EC0DF0070E1F
:10060000506203D0425201E0D57E030E4F622FD0DC
:1006100043A019D174EC15F051C01DF052C01EF06A
:10062000F7EC17F06EEC19F058C037F059C038F0FD
:100630005AC039F05BC03AF05CC03BF084EC19F072
:1006400094C037F095C038F096C039F097C03AF0B2
:1006500098C03BF047EC1AF032C06CF033C06DF03C
:1006600034C06EF035C06FF036C070F00882040EF2
:100670004F6290D05750995DD8B48CD0996714D000
:100680007BC062F07CC063F07DC064F07EC065F02A
:100690007FC066F07BC067F07CC068F07DC069F009
:1006A0007EC06AF07FC06BF0010E996314D080C0E9
:1006B00062F081C063F082C064F083C065F084C0E2
:1006C00066F080C067F081C068F082C069F083C0C6
:1006D0006AF084C06BF0020E996314D085C062F09A
:1006E00086C063F087C064F088C065F089C066F09A
:1006F00085C067F086C068F087C069F088C06AF07E
:1007000089C06BF0030E996314D08AC062F08BC06D
:1007100063F08CC064F08DC065F08EC066F08AC056
:1007200067F08BC068F08CC069F08DC06AF08EC035
:100730006BF0040E996314D09CC062F09DC063F00E
:100740009EC064F09FC065F0A0C066F09CC067F0DA
:100750009DC068F09EC069F09FC06AF0A0C06BF0B9
:1007600099C057F044A40AD08FC062F090C063F0E3
:1007700091C064F092C065F093C066F044AA0AD0BC
:100780008FC067F090C068F091C069F092C06AF0C5
:1007900093C06BF0050E4F6224D007B422D043A063
:1007A0000FD044B20DD0020EC16505D0D00EBB6F84
:1007B000070EBC6F05D0BC6703D0BB5301E1448278
:1007C00043A20FD044B80DD0020EC26505D0D00EA2
:1007D000BD6F070EBE6F05D0BE6703D0BD5301E1EC
:1007E0004488060E4F622FD043A22DD082EC15F024
:1007F00053C01DF054C01EF0F7EC17F06EEC19F06A
:1008000058C037F059C038F05AC039F05BC03AF0E0
:100810005CC03BF084EC19F094C037F095C038F020
:1008200096C039F097C03AF098C03BF047EC1AF008
:1008300032C071F033C072F034C073F035C074F060
:1008400036C075F00882070E4F621FD043A21DD03C
:1008500007A410D04650565CD8B006D0448644BA9F
:100860005768449A8C9205D0449644AA5768448AA3
:100870008C820BD044A805D044AA5768448A8C8245
:1008800004D044BA5768449A8C92080E4F621FD025
:1008900043A01DD007A410D04550555CD8B006D059
:1008A000448044B4576844948C9605D0449044A442
:1008B000576844848C860BD044A205D044A4576862
:1008C00044848C8604D044B4576844948C96090EB2
:1008D0004F6202D08EEC04F00A0E4F6203D04252F7
:1008E00001E0D58E0B0E4F6217D0425215E143A0A6
:1008F00008D0B95306E1428883EC00F043908DECB8
:1009000005F043A208D0BA5306E1428A83EC00F016
:1009100043928DEC05F00882FFEF01F0F8EC11F046
:10092000AD33AC33AD33AC33ACC055F0F6EC11F0B5
:10093000AD33AC33AD33AC33ACC056F01200010E66
:1009400099630AD080C07BF081C07CF082C07DF0CA
:1009500083C07EF084C07FF0020E99630AD085C008
:100960007BF086C07CF087C07DF088C07EF089C0B7
:100970007FF0030E99630AD08AC07BF08BC07CF0B5
:100980008CC07DF08DC07EF08EC07FF01200E8EC50
:1009900017F06EEC19F056EC1CF0EEEC1FF0020EA6
:1009A0003C6E3D6A90EC1FF0E1EC1EF0000EF86E1C
:1009B000290EF76EF00EF66EE7EC11F01200000E45
:1009C000F86E260EF76E440EF66EE3EC11F094C04E
:1009D00032F095C033F096C034F097C035F098C02F
:1009E00036F0EEEC1FF0030E3C6E3D6A90EC1FF00B
:1009F0003F84E1EC1EF0000EF86E260EF76E940EAA
:100A0000F66EE7EC11F0000EF86E260EF76E4E0E45
:100A1000F66EE3EC11F007B009D0000EF86E260E6A
:100A2000F76E5C0EF66EE7EC11F008D0000EF86E73
:100A3000260EF76E600EF66EE7EC11F06FEC10F01C
:100A4000C7EC11F008821200A56708D0000EF86EFE
:100A5000270EF76E280EF66EE3EC11F0010EA5637B
:100A600008D0000EF86E270EF76E3A0EF66EE3EC25
:100A700011F0020EA56308D0000EF86E270EF76E77
:100A80004C0EF66EE3EC11F0030EA56308D0000ED9
:100A9000F86E270EF76E5E0EF66EE3EC11F0040EA4
:100AA000A56308D0000EF86E270EF76E700EF66E76
:100AB000E3EC11F0120083EC00F0000EF86E270E4C
:100AC000F76E160EF66EE3EC11F024EC05F04852CA
:100AD0000FE048AEA52B48BEA507050EA56302D0C2
:100AE000A56B04D0A5AF02D0040EA56F486AEDD760
:100AF000F7EC0FF0ECE311EC10F0040E476203D0BA
:100B000092EC05F005D0050E476202D092EC05F09C
:100B1000C7EC11F0476A0882120043A08C9643A2EA
:100B20008C921200A56702D044EF09F0010EA56374
:100B300003D04380439210D0020EA56303D04390AC
:100B400043820AD0030EA56303D04380438204D0BE
:100B5000040EA56301D003D0E0DF06EC01F0120023
:100B6000A46708D0000EF86E270EF76ECA0EF66E58
:100B7000E3EC11F0010EA46308D0000EF86E270E0E
:100B8000F76EDC0EF66EE3EC11F0020EA46308D0F3
:100B9000000EF86E270EF76EEE0EF66EE3EC11F017
:100BA000030EA46308D0000EF86E280EF76E000E38
:100BB000F66EE3EC11F0040EA46308D0000EF86E9C
:100BC000280EF76E120EF66EE3EC11F0050EA4631C
:100BD00008D0000EF86E280EF76E240EF66EE3ECC9
:100BE00011F0060EA46308D0000EF86E280EF76E02
:100BF000360EF66EE3EC11F0070EA46308D0000E7B
:100C0000F86E290EF76E260EF66EE3EC11F0080E64
:100C1000A46308D0000EF86E290EF76E5C0EF66E17
:100C2000E3EC11F0090EA46308D0000EF86E280E54
:100C3000F76E480EF66EE3EC11F00A0EA46308D0CE
:100C4000000EF86E280EF76E5A0EF66EE3EC11F0F9
:100C50000B0EA46308D0000EF86E280EF76EA20EDD
:100C6000F66EE3EC11F00C0EA46308D0000EF86EE3
:100C7000280EF76E6C0EF66EE3EC11F00D0EA46309
:100C800008D0000EF86E290EF76E920EF66EE3ECA9
:100C900011F0120083EC00F0000EF86E270EF76ED4
:100CA000820EF66EE3EC11F0B0EC05F048520FE066
:100CB00048BE06D0A42B0E0EA46301D0A46B05D0B1
:100CC000A407A4AF02D00D0EA46F486AEDD7F7ECCD
:100CD0000FF0ECE311EC10F0040E476246D0C7ECC5
:100CE00011F0A46701D041D0010EA46302D0DCEF63
:100CF0000AF0020EA46302D004EF0BF0030EA4630B
:100D000002D02CEF0BF0040EA46302D054EF0BF0D2
:100D1000050EA46302D0FFEF09F0060EA46302D013
:100D2000E4EF09F0070EA46302D044EF09F0080EC7
:100D3000A46302D0BCEF0BF0090EA46302D084EFD1
:100D400001F00A0EA46302D054EF08F00B0EA46366
:100D500002D0B4EF07F00C0EA46302D03CEF07F012
:100D60000D0EA46302D0BEEF06F01200440EA2B135
:100D7000430ECFEC11F07AEC11F012009CC00EF192
:100D80009DC00FF19EC010F19FC011F1A0C012F1E3
:100D900083EC00F0A26B000EF86E290EF76EA40E25
:100DA000F66EE3EC11F0000EF86E280EF76EC60E2C
:100DB000F66EE3EC11F09CC032F09DC033F09EC0A3
:100DC00034F09FC035F0A0C036F0EEEC1FF0030EFB
:100DD0003C6E3D6A90EC1FF0E1EC1EF0000EF86EE8
:100DE000260EF76E940EF66EE7EC11F0B6EC06F0F8
:100DF000485223E09CC032F09DC033F09EC034F0D6
:100E00009FC035F0A0C036F09FEC1BF0A2B1AEEC55
:100E10001BF048AE47EC1AF048BE41EC1AF005EC66
:100E200017F032C09CF033C09DF034C09EF035C046
:100E30009FF036C0A0F0486AAED7F7EC0FF0D8E3C9
:100E400011EC10F0040E476203D0BEEC00F011D09C
:100E5000050E476202D0A2719ED70EC19CF00FC151
:100E60009DF010C19EF011C19FF012C1A0F036ECB0
:100E700000F07CEC11F0120007C00EF183EC00F0E2
:100E8000000EF86E280EF76E7E0EF66EE3EC11F093
:100E9000000EF86E280EF76E900EF66EE3EC11F071
:100EA0000E0ECFEC11F0580E07A4200E2AEC11F014
:100EB000F7EC0FF0FDE311EC10F0010E476202D0E9
:100EC0000774DED7040E476203D018EC01F004D09B
:100ED0000EC107F036EC00F01200010E43620AD09A
:100EE000000EF86E280EF76EE20EF66EE3EC11F0CF
:100EF000F8EC11F0020E43620AD0000EF86E280ED4
:100F0000F76EE80EF66EE3EC11F0F6EC11F0AE338E
:100F1000AD33AC33AE33AD33AC3382EC15F0ACC093
:100F20001DF0D6EC1FF0030E3C6EB5EF1EF076C040
:100F300032F077C033F078C034F079C035F07AC041
:100F400036F058C037F059C038F05AC039F05BC09D
:100F50003AF05CC03BF004EC1AF014EC17F013C04C
:100F60009AF014C09BF0120083EC00F09AC04BF191
:100F70009BC04CF19AC01DF09BC01EF0E8EC17F02E
:100F80006EEC19F058C037F059C038F05AC039F03B
:100F90005BC03AF05CC03BF084EC19F005EC17F054
:100FA00032C076F033C077F034C078F035C079F0D5
:100FB00036C07AF0000EF86E280EF76EB40EF66E9C
:100FC000E3EC11F0000EF86E280EF76EC60EF66E0A
:100FD000E3EC11F076C032F077C033F078C034F033
:100FE00079C035F07AC036F0EEEC1FF0030E3C6E9F
:100FF0003D6A90EC1FF0E1EC1EF0000EF86E260E3C
:10100000F76E940EF66EE7EC11F091DF000EF86EBD
:10101000280EF76ECA0EF66EE3EC11F082EC15F0B6
:101020009AC01DF09BC01EF0D6EC1FF0040E3C6E63
:10103000B5EC1EF0485225E076C032F077C033F0B0
:1010400078C034F079C035F07AC036F0400E3B6E8F
:10105000A00E3A6E376A386A396A48AE47EC1AF021
:1010600048BE41EC1AF005EC17F032C076F033C000
:1010700077F034C078F035C079F036C07AF0486A3D
:1010800099D7F7EC0FF0D6E311EC10F0040E47629D
:1010900004D04DDFD0EC00F006D04BC19AF04CC12B
:1010A0009BF036EC00F0120083EC00F045C04BF1F1
:1010B00046C04CF143C04DF1C7D8000EF86E280E63
:1010C000F76ED00EF66EE3EC11F0000EF86E290EFE
:1010D000F76E1A0EF66EE3EC11F0FFDE79EC10F00D
:1010E000F7EC0FF0FAE311EC10F0040E4762A9D010
:1010F000ACC04EF1476A000EF86E280EF76EEE0E89
:10110000F66EE3EC11F0000EF86E290EF76E1A0E73
:10111000F66EE3EC11F0E1DE79EC10F0F7EC0FF095
:10112000FAE311EC10F0040E47628BD0ACC04FF123
:101130004EC11DF04FC122F022501D5CD8B004D02A
:1011400022C04EF11DC04FF174EC15F04EC11DF0E0
:101150004FC122F0F2EC18F0D8901D3289EC15F056
:101160004FC122F007EC19F01DC04EF1000EF86ED1
:10117000290EF76E000EF66EE3EC11F0000EF86E1D
:10118000290EF76E120EF66EE3EC11F082EC15F0FC
:101190004EC11DF0D6EC1FF0030E3C6EB5EC1EF0F8
:1011A000D1EC11F0280E2AEC11F04EC11DF0D2EC5A
:1011B00017F06EEC19F03C0E3B6EA00E3A6EA00ECE
:1011C000396EA00E386E8E0E376E84EC19F0EEEC90
:1011D0001FF0030E3C6E020E3D6E90EC1FF0E1EC32
:1011E0001EF0560E2AEC11F0290E2AEC11F048528E
:1011F0000AE04EC11DF048AE1D2A48BE1D061DC0A6
:101200004EF1486ABBD7F7EC0FF0F1E311EC10F0A8
:10121000040E476210D0010E436205D04EC145F066
:10122000F4EC00F007D0020E436204D04EC146F049
:10123000E2EC00F006D04BC145F04CC146F036EC74
:1012400000F04DC143F01200000EF86E290EF76E4B
:10125000380EF66EE3EC11F0000EF86E290EF76E04
:101260004A0EF66EE3EC11F011EC10F0010E47623D
:1012700003D0010E436E05D0020E476202D0020E6B
:10128000436EC7EC11F0120083EC00F0B0C00EF119
:10129000B1C00FF1B4C013F1B5C014F143C04BF1AC
:1012A000030E436201D0D0DFC7EC11F0000EF86EE0
:1012B000290EF76ECA0EF66EE3EC11F0010E4362D2
:1012C0000DD0000EF86E290EF76EDC0EF66EE3EC14
:1012D00011F0B0C04CF1B1C04DF10FD0020E43621D
:1012E0000CD0000EF86E290EF76EE60EF66EE3ECEB
:1012F00011F0B4C04CF1B5C04DF1480ECFEC11F077
:101300004CC11DF04DC11EF0C7EC04F0485233E053
:1013100074EC15F04CC11DF04DC11EF0640E226E30
:1013200048AE07EC19F048BEF2EC18F0C80E226E79
:10133000000E236E23501E5C02E122501D5CD8B0CB
:1013400005D022C01DF023C01EF00FD0B80E226EB3
:101350000B0E236E1E50235C02E11D50225CD8B0A0
:1013600004D022C01DF023C01EF01DC04CF11EC0D1
:101370004DF1486AC2D7F7EC0FF0C8E311EC10F05A
:10138000040E476214D0010E436207D04CC1B0F086
:101390004DC1B1F03CEC01F014D0020E436207D015
:1013A0004CC1B4F04DC1B5F02AEC01F00AD00EC129
:1013B000B0F00FC1B1F013C1B4F014C1B5F036EC08
:1013C00000F04BC143F01200088444948C9699C0FD
:1013D00050F1040E996F94C032F095C033F096C06E
:1013E00034F097C035F098C036F014EC17F013C005
:1013F000A1F043C04BF1010E436E8C92120083ECBE
:1014000000F0C7EC11F058C027F159C028F15AC0BC
:1014100029F15BC02AF15CC02BF194C02CF195C07E
:101420002DF196C02EF197C02FF198C030F194C0E5
:1014300032F095C033F096C034F097C035F098C0C4
:1014400036F014EC17F013C0A1F0FCEC11F074ECC2
:1014500015F0ACC01DF0ADC01EF0F7EC17F06EEC4F
:1014600019F03F0E3B6E0F0E3A6E760E396E460E39
:10147000386EC40E376E84EC19F094C037F095C006
:1014800038F096C039F097C03AF098C03BF041EC84
:101490001AF0000EF86E260EF76E340EF66EE3ECC0
:1014A00011F0EEEC1FF0030E3C6E3D6A90EC1FF065
:1014B0003F84E1EC1EF0000EF86E260EF76E940EDF
:1014C000F66EE7EC11F0000EF86E290EF76EB60E10
:1014D000F66EE3EC11F082EC15F0A1C01DF0D2EC39
:1014E00017F06EEC19F0EEEC1FF0030E3C6E3D6A47
:1014F0003F8490EC1FF0E1EC1EF0000EF86E260E1B
:10150000F76E940EF66EE7EC11F0000EF86E290EF1
:10151000F76EC00EF66EE3EC11F079EC10F0485265
:1015200014E048AEA12B48BEA107A1C01DF0D2EC2B
:1015300017F02DC094F02EC095F02FC096F030C05B
:1015400097F031C098F0486A80D7F7EC0FF001E2CD
:101550007CD711EC10F0050E476201D0E0D7040EE5
:10156000476213D0A1C01DF0D2EC17F02DC094F04B
:101570002EC095F02FC096F030C097F031C098F093
:101580004EEC01F0A0EC00F016D027C158F028C1B5
:1015900059F029C15AF02AC15BF02BC15CF02CC173
:1015A00094F02DC195F02EC196F02FC197F030C167
:1015B00098F036EC00F01200000EF86E260EF76E72
:1015C000640EF66EE3EC11F0000EF86E260EF76E68
:1015D000760EF66EE3EC11F080C00EF181C00FF1D3
:1015E00082C010F183C011F184C012F185D80EC100
:1015F00080F00FC181F010C182F011C183F012C1DF
:1016000084F072EC01F01200000EF86E260EF76EF8
:10161000640EF66EE3EC11F0000EF86E260EF76E17
:101620007C0EF66EE3EC11F085C00EF186C00FF172
:1016300087C010F188C011F189C012F15DD80EC1C8
:1016400085F00FC186F010C187F011C188F012C17A
:1016500089F072EC01F01200000EF86E260EF76EA3
:10166000640EF66EE3EC11F0000EF86E260EF76EC7
:10167000820EF66EE3EC11F08AC00EF18BC00FF112
:101680008CC010F18DC011F18EC012F135D80EC191
:101690008AF00FC18BF010C18CF011C18DF012C116
:1016A0008EF072EC01F01200000EF86E260EF76E4E
:1016B000640EF66EE3EC11F0000EF86E260EF76E77
:1016C0008E0EF66EE3EC11F08FC00EF190C00FF1AC
:1016D00091C010F192C011F193C012F10DD80EC15A
:1016E0008FF00FC190F010C191F011C192F012C1B2
:1016F00093F072EC01F0120083EC00F00EC132F0B6
:101700000FC133F010C134F011C135F012C136F001
:10171000440ECFEC11F0EEEC1FF0030E3C6E3D6A70
:1017200090EC1FF0E1EC1EF0000EF86E260EF76E46
:10173000940EF66EE7EC11F048520AE0AEEC1BF0A6
:1017400048AE47EC1AF048BE41EC1AF0486AE0D7C0
:10175000F7EC0FF0F1E311EC10F0040E47620AD041
:1017600032C00EF133C00FF134C010F135C011F1A9
:1017700036C012F1476A120007C00EF183EC00F088
:10178000000EF86E290EF76E6E0EF66EE3EC11F099
:10179000000EF86E290EF76E800EF66EE3EC11F077
:1017A000050ECFEC11F0580E07A0200E2AEC11F018
:1017B000450ECFEC11F0580E07A2200E2AEC11F0C6
:1017C000F7EC0FF0FDE311EC10F0010E476202D0D0
:1017D0000770D6D7020E476205D00772D1D718EC32
:1017E00001F00AD0040E476203D018EC01F004D0D7
:1017F0000EC107F036EC00F01200430E3B6E960E61
:101800003A6E376A386A396A76C032F077C033F098
:1018100078C034F079C035F07AC036F012EC1DF0A3
:1018200002E386D801D001D8120064D836BE5FD05A
:10183000430E3B6E160E3A6E376A386A396A12ECFE
:101840001DF005E3520E4D6E030E4E6E52D0420E49
:101850003B6E480E3A6E376A386A396A12EC1DF0F0
:1018600005E3EE0E4D6E020E4E6E43D0410E3B6E02
:10187000A00E3A6E376A386A396A12EC1DF005E339
:10188000F40E4D6E010E4E6E34D0410E3B6E700E56
:101890003A6E376A386A396A12EC1DF005E3FA0EBF
:1018A0004D6E000E4E6E25D0410E3B6E200E3A6EF0
:1018B000376A386A396A12EC1DF005E3C80E4D6EBE
:1018C000000E4E6E16D0400E3B6EA00E3A6E376A7A
:1018D000386A396A12EC1DF005E3460E4D6E000EB3
:1018E0004E6E07D01E0E4D6E000E4E6E02D04D6A2B
:1018F0004E6A120076C037F077C038F078C039F001
:1019000079C03AF07AC03BF05DC032F05EC033F08F
:101910005FC034F060C035F061C036F041EC1AF0C1
:1019200014EC17F013C0C0F0C0AF01D0C06B1200B0
:10193000E1DF36BE5FD0430E3B6E160E3A6E376A5D
:10194000386A396A12EC1DF005E3520E4D6E030E33
:101950004E6E52D0420E3B6E480E3A6E376A386A6F
:10196000396A12EC1DF005E3EE0E4D6E020E4E6E5E
:1019700043D0410E3B6EA00E3A6E376A386A396A20
:1019800012EC1DF005E3580E4D6E020E4E6E34D073
:10199000410E3B6E700E3A6E376A386A396A12EC45
:1019A0001DF005E3F40E4D6E010E4E6E25D0410E76
:1019B0003B6E200E3A6E376A386A396A12EC1DF0B7
:1019C00005E3900E4D6E010E4E6E16D0400E3B6E2E
:1019D000A00E3A6E376A386A396A12EC1DF005E3D8
:1019E0002C0E4D6E010E4E6E07D0C80E4D6E000EC1
:1019F0004E6E02D04D6A4E6A120043A010D007A06E
:101A00000ED052509B5D02E151509A5DD8B005D086
:101A1000B76705D02CEC0DF002D0C80EB76F1200DE
:101A200043B016D0520E1D6E030E1E6E4A501E5C41
:101A300002E149501D5CD8A407D0AF6709D0AE675A
:101A400007D029EC0DF004D0B0C0AEF0B1C0AFF0BB
:101A50001200428067EF00F0428467EF00F043A27B
:101A600010D007A20ED054509B5D02E153509A5DF6
:101A7000D8B005D0B86705D05EEC0DF002D0C80E26
:101A8000B86F120043B216D0520E1D6E030E1E6EBA
:101A90004C501E5C02E14B501D5CD8A407D0B367CC
:101AA00009D0B26707D05BEC0DF004D0B4C0B2F03F
:101AB000B5C0B3F01200428284EF00F0428684EF9A
:101AC00000F083EC00F07FEC10F0425203E083EC76
:101AD00000F086D0F1EC0DF043A040D062C037F0AA
:101AE00063C038F064C039F065C03AF066C03BF0BE
:101AF0006CC032F06DC033F06EC034F06FC035F0A2
:101B000070C036F012EC1DF004E367EC00F0C16B1E
:101B100023D06CC076F06DC077F06EC078F06FC0E7
:101B200079F070C07AF062C05DF063C05EF064C0AE
:101B30005FF065C060F066C061F0FDEC0BF0C0C006
:101B4000C1F04DC049F04EC04AF06CEC00F0526656
:101B500003D0640E516402D0C80EB96F43A240D0C6
:101B600067C037F068C038F069C039F06AC03AF031
:101B70006BC03BF071C032F072C033F073C034F010
:101B800074C035F075C036F012EC1DF004E384EC3F
:101B900000F0C26B23D071C076F072C077F073C0D2
:101BA00078F074C079F075C07AF067C05DF068C0F5
:101BB0005EF069C05FF06AC060F06BC061F0FDEC80
:101BC0000BF0C0C0C2F04DC04BF04EC04CF089ECE1
:101BD00000F0546603D0640E536402D0C80EBA6F8E
:101BE0001200080EA66F516A526A536A546AFCECDE
:101BF00011F0AC515126AD515222FAEC11F0AC511A
:101C00005326AD515422A62FF2D712004250030B97
:101C10000BE0089442B20884000EF86E260EF76EB0
:101C2000BC0EF66EE3EC11F042500C0B0BE0089486
:101C300042B60884000EF86E260EF76EAA0EF66EF7
:101C4000E3EC11F04250300B0BE0089442BA0884E8
:101C5000000EF86E260EF76ECE0EF66EE3EC11F067
:101C6000A22BA2AB09D0000EF86E270EF76E040E61
:101C7000F66EE3EC11F013D008A409D0000EF86E54
:101C8000260EF76EF20EF66EE3EC11F008D0000EA1
:101C9000F86E260EF76EE00EF66EE3EC11F0089487
:101CA0001200EEEC1FF0030E3C6E3D6A90EC1FF04C
:101CB000E1EC1EF0000EF86E260EF76E940EF66E36
:101CC000E7EC11F01200425203E006EC0EF0FCD0FB
:101CD000436611D0000EF86E2A0EF76E100EF66EE7
:101CE000E3EC11F0000EF86E2A0EF76E220EF66E7F
:101CF000E3EC11F0E9D0010E436213D0000EF86E50
:101D0000260EF76E340EF66EE3EC11F06CC032F076
:101D10006DC033F06EC034F06FC035F070C036F077
:101D200015D0020E4362A6D0000EF86E260EF76E96
:101D30003A0EF66EE3EC11F071C032F072C033F07F
:101D400073C034F074C035F075C036F0AADFA32B31
:101D5000A3AF2DD0000EF86E260EF76E980EF66E1D
:101D6000E3EC11F0010E436205D051C01DF052C0EA
:101D70001EF007D0020E436204D053C01DF054C0C1
:101D80001EF0E8EC17F06EEC19F0410E3B6E376A6E
:101D9000386A396A3A6A04EC1AF0EEEC1FF0040E65
:101DA0003C6E3D6A90EC1FF0E1EC1EF01BD0000E83
:101DB000F86E260EF76E9E0EF66EE3EC11F0010E35
:101DC000436207D0B0C01DF0B1C01EF0C7EC04F0F4
:101DD00009D0020E436206D0B4C01DF0B5C01EF09B
:101DE000C7EC04F072D808A409D0000EF86E290ED2
:101DF000F76EC00EF66EE3EC11F066D0000EF86ED2
:101E0000260EF76EA40EF66EE3EC11F0010E43629F
:101E100005D049C04DF04AC04EF007D0020E4362D3
:101E200004D04BC04DF04CC04EF04E6605D04D6610
:101E300003D0B66749D002D0320EB66F4DC01DF048
:101E40004EC01EF0E8EC17F06EEC19F0EEEC1FF04F
:101E5000040E3C6E3D6A90EC1FF0E1EC1EF034D0B5
:101E6000490E82EC15F0C0C01DF0D6EC1FF0B5ECA9
:101E70001EF02AD0030E436227D0000EF86E260E05
:101E8000F76E340EF66EE3EC11F06CC032F06DC0FC
:101E900033F06EC034F06FC035F070C036F001DF43
:101EA000000EF86E260EF76E400EF66EE3EC11F0A3
:101EB00071C032F072C033F073C034F074C035F0CA
:101EC00075C036F0EEDE01D81200030E436201D079
:101ED00035D008A418D0000EF86E290EF76EBC0E8F
:101EE000F66EE3EC11F094C032F095C033F096C07A
:101EF00034F097C035F098C036F0EEEC1FF03F8418
:101F000053EC0EF073D044B403D044BA01D016D0D1
:101F1000A22BA2AB13D0000EF86E260EF76E8E0E1B
:101F2000F66EE3EC11F08FC032F090C033F091C048
:101F300034F092C035F093C036F056D0996713D084
:101F4000000EF86E260EF76E880EF66EE3EC11F0BA
:101F50007BC032F07CC033F07DC034F07EC035F001
:101F60007FC036F041D0010E996313D0000EF86E99
:101F7000260EF76E760EF66EE3EC11F080C032F0AE
:101F800081C033F082C034F083C035F084C036F0B5
:101F90002BD0020E996313D0000EF86E260EF76E4A
:101FA0007C0EF66EE3EC11F085C032F086C033F0A3
:101FB00087C034F088C035F089C036F015D0030EE4
:101FC000996312D0000EF86E260EF76E820EF66E32
:101FD000E3EC11F08AC032F08BC033F08CC034F0E7
:101FE0008DC035F08EC036F051EC0EF012000400BA
:101FF000D89081AE08D081AC06D081AA04D081A847
:1020000002D081B401D0D8801200000E81AE010E42
:1020100081AC020E81AA030E81A8040E81A4050ED4
:10202000120051D8476AF1DF476E7FEC10F0EDDF08
:10203000475CF7E14FEC00F0640EA66F7FEC10F008
:10204000F7EC0FF03DE3A62FF9D74CEC00F00A0EA9
:102050004726C7EC11F00B0E476201D020D00C0EC2
:10206000476201D01CD00D0E476209D0000EF86EF9
:10207000270EF76EB80EF66EE3EC11F019D00E0EC7
:10208000476209D0000EF86E270EF76E820EF66ECC
:10209000E3EC11F00DD00E0E476201D000D0000E1F
:1020A000F86E270EF76E940EF66EE3EC11F008D082
:1020B000000EF86E270EF76EA60EF66EE3EC11F02A
:1020C00079EC10F003D093DFFEE3120090DFFEE224
:1020D00012006DEC10F06FEC10F06FEC10F075EC7E
:1020E00010F075EC10F075EC10F0FA0E10D0C80E70
:1020F0000ED0640E0CD0320E0AD01E0E08D00A0E7E
:1021000006D0050E04D0020E02D0010E00D004004D
:102110000C6EC80E0A6E150E0B6E0A2EFED70B2E15
:10212000FCD70C2EF6D71200700ED36E400E9B6EAD
:102130000F01806A896A0F0E386F0F0E926E816AE6
:102140008A6A000E396FF70E936E826A8B6A000EF0
:10215000946E000E3A6F836A8C6A000E3B6F000E1D
:10216000956E846A8D6A000E3C6F000E966E000EAE
:10217000C16EBF0EC06E000ED06EF00EF26E000E7D
:10218000F16E000EF06E010E9D6E000EA06E470EF9
:10219000D56E310ECD6E000EBA6E000EB16E00011E
:1021A000EC0ED66E1200A66900EE00F0EE6AA62FC5
:1021B000FDD7120079EC10F079EC10F079EC10F00A
:1021C0008B9E8B9A8B9C7BEC10F0200E89EC11F08F
:1021D000800E89EC11F07FEC10F0200E89EC11F0EC
:1021E000800E89EC11F085EC10F0060E7DEC11F0FC
:1021F0000C0E7DEC11F0140E7DEC11F04AEC11F098
:1022000004EC11F0C7EF11F0C7EC11F0000EF86EFE
:102210002A0EF76EA00EF66EE3EC11F0000EF86ECB
:102220002A0EF76EB20EF66EE3EC11F06DEC10F0C4
:10223000000EF86E2A0EF76EC40EF66EE3EC11F087
:10224000000EF86E2A0EF76ED60EF66EE3EC11F065
:102250006FEF10F00D6E98EC11F00D508B8A8B9C87
:102260008B9EF00B89EC11F00D38F00B52D00D6EF7
:102270000D460D460D4698EC11F00D5040097DECD1
:1022800011F0080EA66F0900F5502AEC11F0A62FE8
:10229000FAD71200000EF86E220EF76EB40EF66E2C
:1022A000080EA76FA86BA85137EC11F0A82BA72F29
:1022B000FAD712000102040F1C0C0F001008041EB4
:1022C00007061E000000001F1F000000000C061F74
:1022D0001F060C00000000000000000000000000CD
:1022E00000000000000000000000000000000000EE
:1022F000000000000E0E01D00C0E0D6E98EC11F0D7
:102300000D50F00B8B9A8B9C8B9E89EC11F00D3845
:10231000F00B040083B0010983B2020983B40409FD
:1023200083B608098C6E8B8E2DD88B9E2BD812000D
:102330000400838E27D8958E25D88B9A23D88B8C32
:10234000AA69AA4F0FD01ED83F961CD88B8E1AD8D8
:1023500083AE3F8617D88B9E15D88B8E13D88B9E55
:102360003FA6EFD7959E8B9CC2EF11F000000000B6
:10237000000000000000000000000000000000005D
:102380000000000000000000000000001200010E2C
:10239000B4D7020EB2D7800EB0D7C00EAED7800928
:1023A000ACD7200E57D7A66FD1EC11F0A62FFCD7D3
:1023B00012000E6E0E380EEC00F02AEC11F00E50EA
:1023C0000EEC00F047D70900F550CFEC11F00900F2
:1023D000F55003E02AEC11F0FAD712001D0E0DD0D3
:1023E000190E0BD0150E09D0110E07D00D0E05D009
:1023F000090E03D0050E01D0010EC26EC282C2B218
:10240000FED7C4CFADF0C3CFACF012000400A6B22B
:10241000FDD705C0A9FF06C0A8FFA69EA69CA6845E
:10242000F29EF2BEFDD7550EA76EAA0EA76EA6822B
:1024300008A0F28EA69412000400A6B2FDD705C033
:10244000A9FFA69EA69CA680A8CF06F01200DECF0C
:1024500006F006EC12F0052AA62FF9D723EF00F0BC
:102460001CEC12F006C0DEFF052AA62FF9D71200D9
:10247000EACF04F0E9CF03F0F2A405D0F2948A7613
:10248000EC0ED66E49D0F2A206D0F29281B2482A62
:1024900081A2480641D09EA038D09E90B10ECF6E4A
:1024A000E00ECE6EBC6702D0BB5306E0BB07BB2973
:1024B000D8B4BC07D8B4BB53AF6702D0AE5306E064
:1024C000AE07AE29D8B4AF07D8B4AE53B36702D0C5
:1024D000B25306E0B207B229D8B4B307D8B4B253A6
:1024E000BE6702D0BD5306E0BD07BD29D8B4BE0704
:1024F000D8B4BD53B667B607B767B707B867B807AC
:10250000B967B907BA67BA0707D0A1B8A19804D0CC
:102510009EA202D09E9200D004C0EAFF03C0E9FF51
:102520001100006ED8CF01F0E0CF02F002C0E0FF52
:10253000005001C0D8FF1000000EF86E250EF76E97
:102540005C0EF66EE3EC11F01200000EF86E250E34
:10255000F76E6E0EF66EE3EC11F0120000202020F4
:10256000202020202020202020202020200040206B
:10257000202020202020202020202020202020007B
:1025800000546173746531202020202020202020F9
:102590002000005461737465322020202020202008
:1025A00020202000005461737465332020202020F7
:1025B00020202020200000546173746534202020E6
:1025C00020202020202020000054617374653520D5
:1025D00020202020202020202000005461737465DA
:1025E0003131202020202020202020000054617341
:1025F000746531322020202020202020200000542B
:102600006173746531332020202020202020200099
:102610000054617374653134202020202020202054
:102620002000005461737465313520202020202063
:1026300020202000004C313A0000004C323A0000CB
:1026400009323A00004F66667365743A00004041F3
:1026500044432D436F6E74726F6C3A006175730062
:1026600065696E0000546173742E3420537065697F
:10267000636865726E004054313A00004054323A4B
:1026800000004054333A00004048613A00004042A4
:10269000793A0000DF43000009414443000009503B
:1026A000776D54004950574D00000054656D702EF1
:1026B0002D6D61782E2D4572726F72000050574D4E
:1026C0006D617854696D2E2D4572726F72000053E2
:1026D000656E736F722F4865697A2D4572722E0090
:1026E000402D204C6F65746B6F6C62656E203120DD
:1026F0002D00402D204C6F65746B6F6C62656E20F1
:1027000032202D0040576569746572206D69742010
:10271000546173746500003D3D3D3D204669784D30
:10272000656E75203D3D3D004050776D4D6178549C
:10273000696D6572204564697400404C6F65746B07
:102740006F6C62656E20312045494E00404C6F65CC
:10275000746B6F6C62656E20322045494E00404CB0
:102760006F65746B2E203120752E322045494E0046
:102770004041626272756368202120202020202061
:102780002000003D3D3D3D3D205345545550203DEA
:102790003D3D3D00003D3D205461737465206C61FA
:1027A0006E67203D3D0040205461737465206C6F5E
:1027B000736C617373656E00003D3D3D205761741D
:1027C0006368646F67203D3D3D0040204162627256
:1027D000756368212020202020202000402054659F
:1027E0006D702E20546173746531202020004020CC
:1027F00054656D702E205461737465322020200062
:10280000402054656D702E20546173746533202010
:102810002000402054656D702E205374616E6462F8
:1028200079202000404C6F65746B2E20542E4F662B
:10283000667365742000404C6F65746B2E20542EB7
:102840004F6666205632200040546573742050490C
:10285000437761746368646F670040534554204C4C
:10286000736368722E54726967672E00404C696307
:102870006874736368722E4F4E2F4F464600004CAB
:102880006963687473636872616E6B655B205D0079
:10289000405431206F6E2F6F66665B5434204F4B6F
:1028A0005D0040534554206D61782054656D702E55
:1028B000202020000054656D702E6D61782E5B54D1
:1028C00034204F4B5D0040543A004941443A0000E7
:1028D000002D204C532D5A757374616E6420312085
:1028E0002D00404C313A0000404C323A0000002D9F
:1028F000204C532D5A757374616E642032202D0064
:10290000005472696767657220205B5434204F4B16
:102910005D00404144433A2000004754342057654D
:10292000697465720000405345542050574D6D61E5
:10293000782054696D65720000417573773A4C6B6D
:102940003120546173746520310040417573773ACA
:102950004C6B3220546173746520320040534554EF
:10296000204144432D436F6E74726F6C2000004C05
:102970006B31205B205D205431205434204F4B00BC
:10298000404C6B32205B205D2054322020202020E0
:102990002000404B616C69622E54656D70657261F8
:1029A00074757200004472656867656265725B5495
:1029B00034204F4B5D00404F663A0000404F3A00D4
:1029C000495B5434204F4B5D00000050574D6D6102
:1029D0007854696D65725B53656B5D00404C6F6543
:1029E000746B2E313A00404C6F65746B2E323A0096
:1029F0007300002D205049432D5761746368646F44
:102A000067202D004052657374617274733A000040
:102A1000004B65696E204C6F65746B6F6C62656E00
:102A20002000402D2D2D2D20616B746976212120F1
:102A30002D2D2D00002D2D2053572D426C6F636BD3
:102A4000616465202D004020456E646C6F732053D7
:102A500063686C6569666500003D3D3D2046756EA6
:102A60006B74696F6E203D3D3D00403D20616267A3
:102A70006562726F6368656E21203D00003D3D20F8
:102A80005361766520446174656E203D3D00403D94
:102A90003D2050494320456570726F6D203D3D00DB
:102AA00000534D442D4C6F657473746174696F6E7F
:102AB0003200406D69742032204C6F65746B6F6C0E
:102AC00062656E000046573A312E30332048573A3F
:102AD000312E303020004031302E30332E32312034
:102AE00020444C344A414C0013D806D8186A196A5D
:102AF0001A6A1B6A1C6A1200136A146A156A166A3B
:102B0000176A12001D6A1E6A1F6A206A216A120073
:102B1000F9DF226A236A246A256A266A1200326A69
:102B2000336A346A356A366A12000EC137F00FC153
:102B300038F010C139F011C13AF012C13BF0120067
:102B40000EC132F00FC133F010C134F011C135F0B5
:102B500012C136F0120037C032F038C033F039C03D
:102B600034F03AC035F03BC036F0120032C037F0D6
:102B700033C038F034C039F035C03AF036C03BF0DD
:102B8000120032C00EF133C00FF134C010F135C065
:102B900011F136C012F1120013C132F014C133F03A
:102BA00015C134F016C135F017C136F0120013C14B
:102BB00037F014C138F015C139F016C13AF017C119
:102BC0003BF0120018C132F019C133F01AC134F0D1
:102BD0001BC135F01CC136F0120018C137F019C105
:102BE00038F01AC139F01BC13AF01CC13BF0120099
:102BF0001DC132F01EC133F01FC134F020C135F0C9
:102C000021C136F012001DC137F01EC138F01FC1BE
:102C100039F020C13AF021C13BF0120022C132F05C
:102C200023C133F024C134F025C135F026C136F07C
:102C3000120022C137F023C138F024C139F025C178
:102C40003AF026C13BF0120027C132F028C133F020
:102C500029C134F02AC135F02BC136F0120027C14A
:102C600037F028C138F029C139F02AC13AF02BC118
:102C70003BF0120037C013F138C014F139C015F120
:102C80003AC016F13BC017F1120032C013F133C045
:102C900014F134C015F135C016F136C017F1120029
:102CA00032C018F133C019F134C01AF135C01BF12C
:102CB00036C01CF1120032C01DF133C01EF134C009
:102CC0001FF135C020F136C021F1120032C022F1CF
:102CD00033C023F134C024F135C025F136C026F1CC
:102CE000120032C027F133C028F134C029F135C0B9
:102CF0002AF136C02BF1120013C01DF014C01EF0D3
:102D000015C01FF016C020F017C021F0120013C02C
:102D100022F014C023F015C024F016C025F017C00F
:102D200026F012001DC013F01EC014F01FC015F0D5
:102D300020C016F021C017F01200223623362436A8
:102D40002536263612001D361E361F362036213611
:102D5000120026322532243223322232120021324E
:102D600020321F321E321D32120006D81836193694
:102D70001A361B361C361200133614361536163624
:102D8000173612001C321B321A3219321832120056
:102D9000F9DF1732163215321432133212001DAE1B
:102DA00004D01E681F682068216812001EAE03D080
:102DB0001F682068216812001FAE02D020682168B9
:102DC000120020AE01D02168120040923FBE408226
:102DD0008CDE280E106ED890AFEC16F0C9EC16F011
:102DE00003D8102EF8D71200B8EC20F00A0E0F6EA0
:102DF00000EE13F0EF50E8B6FD0FE8BED00FEE6E18
:102E00000F2EF8D7C5EC20F012003FD817AE09D02E
:102E1000182AD8B4192AD8B41A2AD8B41B2AD8B474
:102E20001C2A7CEC15F035D030D817AE09D0182A02
:102E3000D8B4192AD8B41A2AD8B41B2AD8B41C2A50
:102E400018C013F019C014F01AC015F01BC016F00A
:102E50001CC017F03FBEBDEC1DF0120016D818C004
:102E600013F019C014F01AC015F01BC016F01CC0E6
:102E700017F03FBEBDEC1DF0120007D876EC15F040
:102E800008D003D87CEC15F004D058EC19F04DEFC5
:102E900017F00AEC18F06EEF19F04CD803E175EC5E
:102EA00015F01AD01AD87F0E276E27502B5E2850A7
:102EB0002C5A2BC00FF02B520FE02BBE06D0D8900F
:102EC000B5EC16F00F2EFBD707D00F1E0F2AD890A7
:102ED000C8EC16F00F2EFBD712003F9E31BE3F8E7E
:102EE000319E75EC15F02DC014F02EC015F02FC0DA
:102EF00016F030C017F031C018F0D890B5EC16F0CD
:102F0000C9EC16F0178E18C02BF0186AD890B5ECE3
:102F100016F01200040E0F6EEE6608D00F2EFCD7CE
:102F2000EECFE8FF7F0B03E1D88401D0D894C5EC45
:102F300020F01200B8EC20F000EE2DF0EBD7B8EC4A
:102F400020F000EE32F0E6D7B8EC20F000EE37F0DB
:102F5000E1D7B8EC20F000EE1DF0DCD7B8EC20F0A3
:102F600000EE22F0D7D7B8EC20F000EE13F00A0EF6
:102F70000F6EEE66DBD70F2EFCD7D6D7216A20BEA8
:102F8000216835D0206A216A1FAE31D020682168BF
:102F90002ED01F6A206A216A1EAE29D01F682068C1
:102FA000216825D01E6A1F6A206A216A1DAE1FD0C3
:102FB0001E681F68206821681AD075EC15F03F9EC6
:102FC000216A1DD075EC15F03F9E206A216A17D04A
:102FD00075EC15F03F9E1F6A206A216A10D075ECCF
:102FE00015F03F9E1E6A1F6A206A216A08D075ECA0
:102FF00015F03F9E21AE03D0CCEC1DF03F8E1DC0DE
:1030000018F01EC019F01FC01AF020C01BF021C01C
:103010001CF000D07F0E2B6E000E2C6EB3EC17F060
:1030200006E12D6A2E6A2F6A306A316A36D074EC56
:1030300018F007E0D890C8EC16F02B2AD8B42C2A48
:10304000F6D718B00AD0D890B5EC16F02B062B287E
:10305000D8B42C06D8B42B52F4D714A00BD01480BB
:10306000142AD8B4152AD8B4162AD8B4172AD8B432
:10307000182ADDD7136A18902BC018F0C8EC16F088
:1030800014C02DF015C02EF016C02FF017C030F070
:1030900018C031F0319E3FBE318E12002D6A2E6A6B
:1030A0002F6A316A800E306EF5D72D682E682F6832
:1030B0007F0E306E7F0E316EEDD77F0E1D6E000ECF
:1030C0001E6E2C501E5C02E12B501D5CD8B003D04C
:1030D000ECDFD88401D0D89412002CAE03D0DEDF10
:1030E000D88401D0D8941200B8EC20F000EE1CF087
:1030F000040E0F6EED660AD00F2EFCD7010EEF62A4
:1031000001D002D0EF6602D0D88401D0D894C5ECAB
:1031100020F0120022C000F123C001F124C002F10E
:1031200025C003F126C004F1D4EC18F013C007F158
:1031300014C008F115C009F116C00AF117C00BF14F
:1031400000C11DF001C11EF002C11FF003C120F03B
:1031500004C121F0BAEC18F007C118F008C119F049
:1031600009C11AF00AC11BF00BC11CF03F9E40B20E
:103170003F8E1200BADC280E106ED89005D8BCEC39
:1031800016F0102EFAD71200B8EC20F0050E0F6ED4
:1031900000EE1DF0D890EF50E8200700EE6E0F2EE5
:1031A000FAD7C5EC20F01200B8EC20F09EDC280E17
:1031B000106ED890AFEC16F0C9EC16F000EE1DF0D2
:1031C000050E0F6EEFAE02D0300EEF5EEFA602D00E
:1031D000030EEF5EEE520F2EF5D7102EEAD7C5EC98
:1031E00020F0120002D87CEF16F0B8EC20F09ADD47
:1031F00000EE13F010EE22F0040E0F6EE650EE5EBD
:10320000E650EE5A0F2EFCD7C5EC20F0120002D883
:103210007CEF16F0B8EC20F085DD00EE13F010EE38
:1032200022F0E650EE26040E0F6EE650EE220F2E30
:10323000FCD7C5EC20F0120000C11DF001C11EF04A
:1032400002C11FF003C120F004C121F005C127F025
:1032500006C128F0120007C122F008C123F009C1FD
:1032600024F00AC125F00BC126F00CC129F00DC1D4
:103270002AF0120014C000F115C001F116C002F1CD
:1032800017C003F118C004F12BC005F12CC006F1E2
:10329000120014C007F115C008F116C009F117C0DB
:1032A0000AF118C00BF12BC00CF12CC00DF112006B
:1032B00032C02DF033C02EF034C02FF035C030F0C6
:1032C00036C031F0120037C02DF038C02EF039C0B2
:1032D0002FF03AC030F03BC031F012002DC032F078
:1032E0002EC033F02FC034F030C035F031C036F08E
:1032F00012002DC037F02EC038F02FC039F030C08A
:103300003AF031C03BF01200D5EC20F016E2D2ECDE
:1033100020F013E29FEC17F01AE0A4EC17F017E08E
:10332000EAEC20F004E39FEC17F001E306D0EDECAB
:1033300020F006E3A4EC17F003E312EC21F01200F6
:10334000EAEC20F003E307EC21F003D00DD08FEC82
:1033500015F036BE03D03BAE01D0368E36AE03D06C
:103360003BBE01D0368E12001DD83F9E3FBA3F7E35
:103370003FBC3F7E79EC1DF017C000F118C001F191
:1033800019C002F11AC003F11BC004F11ED80AECE7
:1033900019F07CEC16F089EC15F07F0E226EF5EC3E
:1033A00018F01ED03F9A3F9C36BE3F8A3BBE3F8CF2
:1033B0007FDF6DEC17F05EDF86DF6DEC17F069DF05
:1033C00074EC15F039DF2BEF19F074EC15F027C011
:1033D0001DF028C01EF029C022F02AC023F01200E0
:1033E00013C02BF014C02CF075EC15F000C114F0D4
:1033F00001C115F002C116F003C117F004C118F0A5
:103400000EEC18F06EEF19F0D5EC20F009E2D2ECDA
:1034100020F006E29FEC17F006E1A4EC17F019E1AA
:1034200012EC21F01200EDEC20F003E3EAEC20F0C6
:10343000F7E2A4EC17F010E107EC21F036BE03D060
:103440003BAE01D0368E36AE03D03BBE01D0368EB9
:1034500012001CEC21F0F2D7A5DF3F9E3FBA3F7E61
:103460003FBC3F7E47EC1EF005DFAFDFF5EC18F008
:103470007CEC16F089EC15F07F0E226E0AEC19F048
:10348000AFD7A4EC17F001E112003B7E00D0D5ECE1
:1034900020F004E2D2EC20F001E203D012EC21F0A3
:1034A0001200A4EC17F001E112009FEC17F003E109
:1034B000ABEC15F0120017D80AEC19F027C02BF06E
:1034C00028C02CF03F9E17AE03D03F8EBDEC1DF000
:1034D00013C000F114C001F115C002F116C003F1D0
:1034E00017C004F181D75EDFFE0E2B6E000E2C6E2E
:1034F0002A50285C02E12950275C27E013E3292A9F
:10350000D8B42A2A2C502A5C02E12B50295C07E10E
:1035100089EC15F027C029F028C02AF016D0D890E1
:1035200018DCE6D7272AD8B4282A2C50285C02E1D8
:103530002B50275C07E182EC15F029C027F02AC048
:1035400028F003D0D8900BDCD3D73FBACCEC1DF0D9
:103550003FBCDBEC1DF01200B6EC15F084EF19F067
:103560009FEC17F02DE036BE2CD0D5EC20F028E2F1
:10357000C1EC15F0ECD848DF45EC16F01E0E126ECB
:10358000124E1ED0A0EC15F0D7EC15F03DDFD7ECB5
:1035900015F07DDFDCD838DFD7EC15F03B50365C1A
:1035A0000BE13A50355C08E13950345C05E13850A4
:1035B000335C02E13750325C03E045EC16F0E0D7B3
:1035C000120012EC21F012009FEC17F008E13F0E00
:1035D000366E800E356E326A336A346A120001012B
:1035E0003F0E266F800E256F226B236B246B3F0EE0
:1035F000216F800E206F1D6B1E6B1F6B000150EC46
:1036000016F045EC16F022C10EF123C10FF124C1D2
:1036100010F125C111F126C112F11E0E126ECCEC73
:1036200015F003EC16F0F0DE95EC15F047EC1AF00F
:1036300095EC15F03B50365C0BE13A50355C08E1F7
:103640003950345C05E13850335C02E13750325C6C
:1036500017E0124E15D0C1EC15F00EEC16F06FD835
:1036600016DF66EC16F003EC16F04EDE5BEC16F09F
:10367000E2EC15F0D7EC15F047DE45EC16F0CFD7AD
:1036800012009FEC17F008E13F0E366E800E356E8B
:10369000326A336A346A120032C02CF133C02DF121
:1036A00034C02EF135C02FF136C030F13DEC17F0AB
:1036B0003BD82ADE89DF71EC16F02CC132F02DC127
:1036C00033F02EC134F02FC135F030C136F045EC67
:1036D00017F03F943FBE3F8418C012F027C132F06C
:1036E00028C133F029C134F02AC135F02BC136F09E
:1036F000125206E03FA4C5D83FB4D5D8122EFAD74F
:103700001200420E3B6E480E3A6E376A386A396ACA
:103710001200400E3B6E490E3A6E0F0E396EDA0EF5
:10372000386EA20E376E1200400E3B6E130E3A6ECC
:103730005D0E396E8D0E386EDE0E376E12003F0E46
:103740003B6E800E3A6E376A386A396A1200400E54
:103750003B6E376A386A396A3A6A1200410E3B6E2C
:10376000200E3A6E376A386A396A1200420E3B6E92
:10377000C80E3A6E376A386A396A1200440E3B6ED8
:103780007A0E3A6E376A386A396A1200460E3B6E14
:103790001C0E3A6E400E396E376A386A1200470EB8
:1037A0003B6EC30E3A6E500E396E376A386A12009D
:1037B000490E3B6E740E3A6E240E396E376A386AC3
:1037C00012004B0E3B6E180E3A6E960E396E800E3E
:1037D000386E376A12004C0E3B6EBE0E3A6EBC0E4F
:1037E000396E200E386E376A12004E0E3B6E6E0E2A
:1037F0003A6E6B0E396E280E386E376A12003D0E27
:103800003B6ECC0E3A6ECC0E396ECC0E386ECD0EB1
:10381000376E12003C0E3B6E230E3A6ED70E396E99
:103820000A0E386E3D0E376E12003A0E3B6E830E56
:103830003A6E120E396E6E0E386E980E376E12009A
:10384000350E3B6E860E3A6E370E396EBD0E386EF3
:10385000060E376E1200300E3B6E890E3A6E700EF9
:10386000396E5F0E386E410E376E12002B0E3B6EB6
:103870008C0E3A6EBC0E396ECC0E386E090E376E59
:1038800012006CDF84EF19F071DF84EF19F076DF3E
:1038900084EF19F07BDF84EF19F081DF84EF19F0FA
:1038A00087DF84EF19F05ADF04EF1AF05FDF04EFCF
:1038B0001AF064DF04EF1AF069DF04EF1AF06FDF2B
:1038C00004EF1AF075DF04EF1AF09FEC17F003E134
:1038D00012EC21F01200C1EC15F001013F0E176F40
:1038E000800E166F136B146B156B000128DF41EC13
:1038F0001AF050EC16F0A0EC15F021DF47EC1AF0AE
:103900005BEC16F0E2EC15F003EC16F004EC1AF0A8
:1039100050EC16F066EC16F0C1EC15F0280E126EA5
:10392000CCEC15F014DF47EC1AF045EC16F0E2ECA5
:1039300015F019EC16F084EC19F019EC16F084EC83
:1039400019F050EC16F0D7EC15F004EC1AF095ECE9
:1039500015F047EC1AF095EC15F03B50365C0BE196
:103960003A50355C08E13950345C05E13850335C3D
:1039700002E13750325C05E0124E03D0C1EC15F085
:10398000CFD7E5DE84EF19F00101276B0001AEEC23
:103990001BF048D806E353EC1CF00101272B000173
:1039A000F6D793DFC1DE04EC1AF074EC15F027C1F2
:1039B00018F0185206E00AEC18F079EC19F047EC10
:1039C0001AF012007ED821AE14D026AE29D05AD8D3
:1039D0002150265C0BE12050255C08E11F50245C3F
:1039E00005E11E50235C02E11D50225CD8B016D0C8
:1039F00017D021BE02D026BE11D044D82150265C5B
:103A00000BE12050255C08E11F50245C05E11E50AD
:103A1000235C02E11D50225CD8B002D0D89001D0C6
:103A2000D88012004ED821AE14D026AE29D02AD884
:103A30002150265C0BE12050255C08E11F50245CDE
:103A400005E11E50235C02E11D50225CD8B016D067
:103A500017D021BE02D026BE11D014D82150265C2A
:103A60000BE12050255C08E11F50245C05E11E504D
:103A7000235C02E11D50225CD8B002D0D88001D076
:103A8000D89012009FEC17F003E182EC15F00FD0F4
:103A9000D890A3EC16F0D89020321F321E321D327F
:103AA000208EA4EC17F003E189EC15F009D0D89032
:103AB0009DEC16F0D8902532243223322232258E06
:103AC000120032C01DF033C01EF034C01FF035C0EC
:103AD00020F036C021F037C022F038C023F039C0C2
:103AE00024F03AC025F03BC026F0120002D87CEF4B
:103AF00016F0B8EC20F037D8050E0F6E00EE22F06D
:103B000020EE13F075EC15F010EE1DF0050E106EA2
:103B10000FC011F01050112611061106EF50E602E9
:103B2000F350DE26D9CF3CF0DACF3DF0F450DE2260
:103B3000E86ADE22112EFCD73CC0D9FF3DC0DAFF77
:103B4000102EE6D7EE5220EE13F0060E116E0F5037
:103B5000115EDE52112EFDD70F2ED6D7C5EC20F008
:103B60003FB20BD812003F9221AE02D015D83F725F
:103B700026AE02D020D83F721200131E141E151E4E
:103B8000161E171E132AD8B4142AD8B4152AD8B46E
:103B9000162AD8B4172A12001D1E1E1E1F1E201E14
:103BA000211E1D2AD8B41E2AD8B41F2AD8B4202A10
:103BB000D8B4212A1200221E231E241E251E261ED2
:103BC000222AD8B4232AD8B4242AD8B4252AD8B48F
:103BD000262A1200C8DFB8EC20F075EC15F0050EAF
:103BE0000F6E00EE22F0EE6605D00F2EFCD7C5EC6E
:103BF00020F012000F6A0F2AD89026BE1CD0223661
:103C000023362436253626362650215C0BE12550F6
:103C1000205C08E124501F5C05E123501E5C02E19A
:103C200022501D5CE8E275EC15F0D8902632253262
:103C30002432233222322650215C0BE12550205CB5
:103C400008E124501F5C05E123501E5C02E1225074
:103C50001D5C0AE322501D5E23501E5A24501F5A39
:103C60002550205A2650215ABCEC16F00F2EDDD7D5
:103C700077DF1DC022F01EC023F01FC024F020C03B
:103C800025F021C026F07CEC16F0C5EF20F0290EBF
:103C90000F6E75EC15F02650215C0BE12550205C71
:103CA00008E124501F5C05E123501E5C02E1225014
:103CB0001D5C0BE322501D5E23501E5A24501F5AD8
:103CC0002550205A2650215AD880B5EC16F0D890AD
:103CD000A3EC16F02650215C0BE12550205C08E196
:103CE00024501F5C05E123501E5C02E122501D5C44
:103CF0000BE322501D5E23501E5A24501F5A25509C
:103D0000205A2650215AD8800F2EDFD71200B8EC47
:103D100020F03F9221AE02D03FDF3F8275EC15F0DC
:103D2000280E0F6E0A0E106E00EE13F0EF500F0B00
:103D3000116E050E115CD8A002D0030EEF26EF50D5
:103D4000F00B116E500E115CD8A002D0300EEF2691
:103D5000EC52102EEBD7D890A3EC16F0B5EC16F081
:103D60000F2EE0D7C5EC20F01200D5EC20F015E2C4
:103D7000EDEC20F01CE22FD844D85AD84094120021
:103D8000030E3C6409D03D663C2A3FB43C2A030E36
:103D90003C5E3C50D3EC11F01200F2DF000EF86EE6
:103DA000420EF76E4A0EF66EE7EC11F01200E8DFF5
:103DB000000EF86E420EF76E4E0EF66EE7EC11F046
:103DC0001200D5EC20F0E9E2EDEC20F0F0E203D8AF
:103DD0002FD840941200B8EC20F000EE1CF011EE49
:103DE00031F00A0E116EEDCF0FF00F38106E56D86D
:103DF0000FC010F053D8112EF6D7E76AC5EC20F0AB
:103E00001200B8EC20F03D5210E001EE44F011EE4B
:103E100044F0140E0F6E3DC010F0E5500F06102E4A
:103E2000FCD7E5CFEDFF0F2EFCD7C5EC20F012003C
:103E3000B8EC20F00A0E106E3D5010263C50105C7D
:103E4000D8B002D010C03CF03C503D5CD8A003D0AC
:103E50003DC03CF03C2A3D503C5E3C06090E0F6ED6
:103E60003C500F5E01EE31F00F5204E0EECFE8FF60
:103E70000F2EFCD73FA405D02B0E3FBE2D0E8DEC90
:103E80001FF03F8019D83F9013D83D5204E02C0E0C
:103E90008DEC1FF009D8C5EC20F0120010500F0B6C
:103EA0003009E8CFE6FF12003DC011F0409606D081
:103EB000010E116E409602D03CC011F0115226E066
:103EC0003FA006D0EFCF0FF0300E0F5CD8A43F908C
:103ED00040A611D011C01DF0020E1D6202D087EC69
:103EE0001FF0050E1D6202D087EC1FF0080E1D6248
:103EF00002D087EC1FF0EECFE8FF3FB003D08DEC8F
:103F00001FF002D089EC1FF0112EDAD71200200E1C
:103F100004D0200E40B4300E00D02AEC11F0120074
:103F2000B8EC20F00A0E0F6E3D500F5E00EE13F05D
:103F3000EF500F4E0CD0EF500F4E02D0EE52F8D78C
:103F4000EE521D6E490E1D6409D0010E06D00F0BF6
:103F50001D6E040E1D6402D0100EEF260A0E0F6EA9
:103F600000EE13F0EF500700EE6EE86AEF220F2E1E
:103F7000F9D7C5EC20F01200B8EC20F0050E0F6E5A
:103F80000A0E106E00EE1CF0EDCF1DF01D50F00B70
:103F900007E110061D500F0B03E110060F2EF4D79A
:103FA00010C01DF01050C5EC20F012001CEC21F0E8
:103FB00075EC15F087EC1EF013C018F014C019F062
:103FC00015C01AF016C01BF017C01CF0050E3C6E91
:103FD0003D6A3F9440943F9840961200D5EC20F003
:103FE00044E2EDEC20F041E258EC19F04DEC17F012
:103FF00013C000F114C001F115C002F116C003F1A5
:1040000017C004F118C01DF019C01EF01AC01FF02F
:104010001BC020F01CC021F087EC1EF013C007F17C
:1040200014C008F115C009F116C00AF117C00BF150
:1040300000C11DF001C11EF002C11FF003C120F03C
:1040400004C121F0E5EC16F007C118F008C119F021
:1040500009C11AF00AC11BF00BC11CF0140E3C6E12
:104060000A0E3D6E3F98409640943F941200C1EC7A
:1040700015F03E6A369E9FEC17F014E0AEEC1BF094
:1040800012EC1DF001E004E353EC1CF03E2AF6D7DD
:104090009FEC1BF0E2EC1CF005E004E341EC1CF0AB
:1040A0003E06F6D7EEEC1FF0A0EC15F036BE3F8EC4
:1040B0000B0E3C6E0A0E3D6E3F843F981200E1EC01
:1040C0001EF0650E8DEC1FF03F9E3EBE3F8E3EBE45
:1040D0003E6C82EC15F03EC01DF0D6EC1FF03F8424
:1040E0004BDF1DC03CF0E1EC1EF01200CCEC15F0F3
:1040F00095EC15F041EC1AF071EC16F0F8EC15F0B7
:10410000EDEC15F041EC1AF0B6EC15F027C132F0E9
:1041100028C133F029C134F02AC135F02BC136F063
:1041200004EC1AF071EC16F00EEC16F0EDEC15F054
:1041300041EC1AF02FEC16F084EC19F095EC15F028
:1041400047EC1AF01200B8EC20F082EC15F0050EE6
:104150000F6E10EE13F020EE1DF0E6500F0BDF6E29
:10416000E638F00BDE120F2EF8D7C5EC20F0120067
:10417000E9CF45F1EACF46F1E1CF47F1E2CF48F18F
:10418000D9CF49F1DACF4AF1120045C1E9FF46C162
:10419000EAFF47C1E1FF48C1E2FF49C1D9FF4AC177
:1041A000DAFF120063EC19F003D058EC19F000D0DC
:1041B000319E7F0E31620CD0800E306207D02F66A8
:1041C00005D02E6603D02D6601D002D0D88001D054
:1041D000D890120063EC19F003D058EC19F000D01D
:1041E000319E7F0E31620BD0800E306208D02F6678
:1041F00006D02E6604D02D6602D0D88001D0D8908B
:10420000120002D86EEF19F005D8318E120002D8D4
:104210006EEF19F07F0E316E800E306E2D6A2E6AB1
:104220002F6A120002D86EEF19F07F0E316E2D68E2
:104230002E682F683068120002D86EEF19F02D6AD0
:104240002E6A2F6A306A316A12002D2D2D00494ED8
:02425000460026
:020000040030CA
:0300010028192398
:020005003D803C
:0200000400F00A
:100000000000009B43000000AF43000000B9430024
:100010000000A042000000F0C1012C0120033207C3
:0A0020008080AB1900000037430197
:00000001FF
